:060000000A128A110E280D
:10000800FE00030EF6000408F7000A08F8000A12BA
:100018008A11BC2D0A128A1111280C30FB000130FC
:10002800FC002030831384004A300A128A116F279B
:10003800FD0183010A128A11E32BD10064305102B9
:10004800031808000A30CA00510894230A128A11BA
:10005800D0000A30CA00510879230A128A11CF0049
:100068004F0EF039D00744230A128A11D0309D224E
:100078000A128A1106309D220A128A1150089D22FE
:100088000A128A11522BD1005108031908000D30A9
:100098005102031808000A30CA00510894230A12B2
:1000A8008A11D0000A30CA00510879230A128A112D
:1000B800CF004F0EF039D00744230A128A11D030EE
:1000C8009D220A128A1105309D220A128A115008AF
:1000D8009D220A128A11522BD100510803190800D7
:1000E80020305102031808000A30CA00510894232E
:1000F8000A128A11D0000A30CA00510879230A125C
:100108008A11CF004F0EF039D00744230A128A1102
:10011800D0309D220A128A1104309D220A128A11B7
:1001280050089D220A128A11522BD2003C305202EA
:10013800031808000A30CA00520894230A128A11C8
:10014800D1000A30CA00520879230A128A11D00055
:10015800500EF039D10744230A128A11D0309D225B
:100168000A128A11C12807309D220A128A11C6284C
:1001780000309D220A128A11C6284F08013A031935
:10018800B728BC2851089D220A128A11522B003028
:100198005F210A128A11DA0000305B220A128A11E2
:1001A800FA0000301D220A128A11F900E5200A120D
:1001B8008A11DB0036210A128A11D7000D21D800D6
:1001C800080044230A128A11D0309D220A128A118B
:1001D80006309D220A128A1166230A128A11D1302A
:1001E8009D220A128A110130DB220A128A11D000DC
:1001F80052230A128A115008CF000F30CF05D00EB3
:10020800D005D0050A30CA005008B023CF074F08E0
:10021800080044230A128A11D0309D220A128A113A
:1002280005309D220A128A1166230A128A11D130DA
:100238009D220A128A110130DB220A128A11D0008B
:1002480052230A128A115008CF000F30CF05D00E62
:10025800D0050130D0050A30CA005008B023CF07B6
:100268004F08080044230A128A11D0309D220A122E
:100278008A1104309D220A128A1166230A128A11F1
:10028800D1309D220A128A110130DB220A128A110A
:10029800D00052230A128A115008CF000F30CF0520
:1002A800D00ED0050330D0050A30CA005008B0235C
:1002B800CF074F0808008312CF0044230A128A117F
:1002C800D0309D220A128A11732907309D220A1202
:1002D8008A11782900309D220A128A1178294F083C
:1002E800013A031969296E2966230A128A11D13045
:1002F8009D220A128A110130DB220A128A11D100CA
:1003080052230A128A115108D0000F30D005D10E9D
:10031800D1050730D1050A30CA005108B023D007EB
:1003280050080800D2003C305202031808000A3076
:10033800CA00520894230A128A11D1000A30CA004E
:10034800520879230A128A11D000500EF039D107C9
:1003580044230A128A11D0309D220A128A11C32915
:1003680008309D220A128A11CB290B309D220A12CD
:100378008A11CB2901309D220A128A11CB294F08F4
:10038800013A0319B429033A0319B929BE295108B6
:100398009D220A128A11522BD3003C3053020318B3
:1003A80008004F0BE7290C305302031CE429603086
:1003B800D2000D305302031CE829F430D307E82992
:1003C8004030D200E829D2010A30CA0053089423E9
:1003D8000A128A11D2070A30CA00530879230A126E
:1003E8008A11D100510EF039D20744230A128A111A
:1003F800D0309D220A128A11102A09309D220A1231
:100408008A11182A0C309D220A128A11182A0230E1
:100418009D220A128A11182A5008013A0319012A42
:10042800033A0319062A0B2A52089D220A128A1136
:10043800522BCF0044230A128A11D0309D220A126F
:100448008A11352A08309D220A128A113D2A0B305A
:100458009D220A128A113D2A01309D220A128A1110
:100468003D2A4F08013A0319262A033A03192B2A71
:10047800302A66230A128A11D1309D220A128A1163
:100488000130DB220A128A11D10052230A128A1182
:100498005108D0000F30D005D10ED1050730D10555
:1004A8000A30CA005108B023D00750080800CF000E
:1004B80044230A128A11D0309D220A128A11732A03
:1004C80009309D220A128A117B2A0C309D220A12B9
:1004D8008A117B2A02309D220A128A117B2A4F0830
:1004E800013A0319642A033A0319692A6E2A662312
:1004F8000A128A11D1309D220A128A110130DB2298
:100508000A128A11D10052230A128A11511F912A04
:10051800D2230A128A110130952AD2230A128A118B
:100528000330D1050A30CA005108B023D00750085B
:100538000800CC008030CD01CE004E080319C22A35
:100548004C084E050319AB2A83160516AF2A8316E5
:10055800051283120512013019230A128A11831613
:100568008516013019230A128A11851EB92A8316A5
:100578008512831285120310CE0CA12A8316051644
:10058800013019230A128A1183168516013019239E
:100598000A128A11831605168312051ED52ACD0163
:1005A800CD0A83168512831285124D080800CC00E7
:1005B800CD0183160516013019230A128A118030DD
:1005C800CE004E080319012B831685160130192316
:1005D8000A128A11851EEE2A8316051683124E0802
:1005E800051ACD048316851283128512013019234A
:1005F8000A128A110310CE0CE52A4C080319072B9E
:10060800831605160B2B831605128312051201306B
:1006180019230A128A1183168516013019238316A5
:100628008512831285124D0808008312CB006430AE
:100638004B02031C362BA53083120313CA00CA0BC6
:10064800232B262B643083120313CB021B2B0F3072
:1006580083120313CA00CA0B2F2B322B0A308312C2
:100668000313CB020A304B02031C3E2B2B2B3C2BD3
:100678003D2B000083120313CB034B0F3B2B0800C9
:10068800831685160516013019230A128A11D923F3
:100698000A128A1119230A128A11DE2B831685126F
:1006A80083128512D9230A128A1119230A128A1170
:1006B80083168516013019230A128A118316051626
:1006C8000A30BE2B83160516013019230A128A1127
:1006D80083168516013019230A128A11D9230A12A2
:1006E8008A1119230A128A11DE2BCB00CD014A0880
:1006F8000319922BCC01CC0ACA1B852B0310CA0DF7
:100708007F2B0310CD0D4A084B02031C8F2B4A0880
:10071800CB024D140310CA0CCC0B852B4D080800D6
:10072800CC000830CD00CE014C08CB0007300310B8
:10073800CB0CFF3E0310031D9C2B4E0D4B04CE002B
:100748000310CC0D4A084E02031CAC2B4A08CE02FB
:10075800CD0B982B4E080800CC00CB014A084C184A
:10076800CB070310CA0D0310CC0C4C08031DB22B89
:100778004B0808008312CC0083120313CC034C0FE0
:10078800C62B0800073083120313CB007C30CA0045
:10079800CA0BCC2BCB0BCC2B0000C02B5108D000A4
:1007A8000F30D005D10ED10508008316051283122B
:1007B800051201348316851283128512080007304A
:1007C80083169F00C030810040308312AE00803015
:1007D800AF000130A2000230A3000430A4000830AA
:1007E800A5001030A6002030A7004030A8008030B7
:1007F800A9000B1712109210121512080739383871
:100808009200F930831692008B178C148312CE0154
:10081800CF010A128A1145270A128A114E08FB00D5
:10082800CE01CE0ACF010A128A1145270A128A116F
:100838004E08FC000A128A1177270A128A110A1236
:100848008A11CB200A128A110530CA008530CB01E3
:10085800CC00CD01CE01CE0ACF014C08840083170D
:100868004D1C831300084E04D0004C0884008317E5
:100878004D1C8313500880004A08840083174B1CC2
:10088800831300084E05D0004F0A4C2C0310D00CDF
:10089800FF3E031D4A2C5008DC000530CA00853095
:1008A800CB01CC000230CD01CE00CF01CF0A4C08DD
:1008B800840083174D1C831300084E04D0004C0895
:1008C800840083174D1C8313500880004A08840055
:1008D80083174B1C831300084E05D0004F0A762C53
:1008E8000310D00CFF3E031D742C5008D9005C087F
:1008F80003198F2D330B812C8F2D3208013EB20046
:100908000130B3008F2D59080319A12C330B8D2CFE
:10091800A12C7A08013EFA00B6250A128A11D021C4
:100928000A128A1118307A02031CA12CFA01B62582
:100938000A128A11D0210A128A11B101A92D590867
:100948000319A12C330BA92CA12C7908013EF9001D
:100958003C3079020318F901DA010130B300CF0104
:1009680079080A128A1196210A128A110030CF01D9
:100978000A128A1199200A128A11A12C59080319FE
:10098800D72C330BC82CD72C5B08013EDB00643016
:100998005B020318DB010130B3005B080A128A11FD
:1009A80021200A128A110130882D59080319D72CE1
:1009B800330BDF2CD72C5808013ED8000D305802D5
:1009C80001300318D800B30058080A128A114720CA
:1009D8000A128A11D72C59080319D72C330BF52C76
:1009E800D72C5708013ED700203057020130031892
:1009F800D700B30057080A128A1170200A128A1108
:100A0800D72C590803192B2D330B0B2D162D7B08CA
:100A1800013EFB000130B30018307B02031C162D89
:100A28000C30FB00CF01D0017B08D100D2010A12A3
:100A38008A1113270A128A1183120313CE01CF01D8
:100A48000A128A1145270A128A114E08FB0004303F
:100A5800882D59080319552D330B332D3E2D7C084D
:100A6800013EFC000130B3000D307C02031C3E2D1A
:100A78000130FC00CF01CF0AD0017C08D100D2019F
:100A88000A128A1113270A128A1183120313CE013C
:100A9800CE0ACF010A128A1145270A128A114E0876
:100AA800FC000530882DB201A92D7B08FF3EAF253B
:100AB8000A128A11D60080305602031D652D7A0865
:100AC8005402031C752D7C08FF3E83120313AF25C7
:100AD8000A128A11803C031D732D54087A020318E8
:100AE800792D033083120313882D0A3079060319F0
:100AF800812D28307906031D8A2D1F308312031398
:100B08005A020318A12C0230B100A92D8312031335
:100B1800590BA12CD72C3208013A0319872C033A18
:100B28000319A32C013A0319C22C073A0319D92C2B
:100B3800013A0319EF2C033A0319052D013A031959
:100B48002D2D0F3A0319572D592D5C085904031DF3
:100B5800232CB301232CD400FF3003180030D50018
:100B6800803A08000130B300CF01D0017A080800AC
:100B7800831203138C1CC52D83168C1CC52DCE2502
:100B88008C1078088A0077088400760E8300FE0EA1
:100B98007E0E09007D08013EFD00892E0A30F00016
:100BA8005B08F8260A128A118312B4002030322E0C
:100BB8000A30F0005B08DC260A128A118312B4009E
:100BC8001030322E0A30F0005808F8260A128A111E
:100BD8008312B4000830322E0A30F0005808DC26A0
:100BE8000A128A118312B4000430322E0A30F0003F
:100BF8005708F8260A128A118312B4000230322EDE
:100C08000A30F0005708DC260A128A118312B40051
:100C18000130322EFD01B401B5019B2E7D08023A48
:100C28000319D22D063A0319DC2D023A0319E62DD1
:100C38000E3A0319F02D023A0319FA2D063A031950
:100C4800042E023A03190E2E9B2E0A30F0005A0881
:100C5800DC260A128A118312B4003F30B5009B2E9D
:100C68000A30F0007B08D52D0A30F0007B08DF2D14
:100C78007D08023A0319342E063A0319382E023A2F
:100C880003190E2E9B2E0A30F0007C08FD2D0A3029
:100C9800F0007C08072E7D08023A0319472E063A11
:100CA80003194B2E023A03190E2E9B2E0A30F00020
:100CB8007A08D52D0A30F0007A08DF2D0A30F000C6
:100CC8007908E92D0A30F0007908F32D0A30F00090
:100CD8005A08FD2D0A30F0005A08072E7D08023AFE
:100CE80003195A2E063A03195E2E023A0319622E88
:100CF8000E3A0319662E023A03196A2E063A0319A8
:100D08006E2E023A03190E2E9B2E83123108013AD9
:100D18000319122E033A0319292E013A03199D2E9D
:100D2800073A03193C2E013A03194F2E722E7D1CE7
:100D3800A62E8316870183128701831686018312E4
:100D48008601CE2E02303402031CB42E831686018F
:100D580083123408203E8400831300088600C32EC3
:100D68003F3083168705831234082E3E8400C03036
:100D780083130005F50007083F3975048700C03064
:100D8800831687053F3083123505F5000708C039FB
:100D9800750487005A1CD52E831685118312851178
:100DA8000800831685118312050808388500080095
:100DB800F2000830F300F4017208F1000730031064
:100DC800F10CFF3E0310031DE42E740D7104F400B2
:100DD8000310F20D70087402031CF42E7008F4025C
:100DE800F30BE02E74080800F100F30170080319F2
:100DF800112FF201F20AF01B042F0310F00DFE2E42
:100E08000310F30D70087102031C0E2F7008F10215
:100E180073140310F00CF20B042F73080800500829
:100E2800CB004F08CA005208CD005108CC001C2F37
:100E3800831603178C181C2F831203134A080317F1
:100E48008D0003134C0803178C0083168C130C15A4
:100E580000308B1B013083120313CE008B135530E7
:100E6800831603178D00AA308D008C148C183A2F26
:100E7800831203134E08031D8B17831603170C11D7
:100E880008004F08CB004E08CA0053274B08D10072
:100E98004A08D0005108CF005008CE0008004A0880
:100EA80003178D0083168C130C1483120C0803137C
:100EB800CC00CD014D08CB004C08CA000800073013
:100EC8008A000408840A820700342F34003430343E
:100ED80000343A34003464008001840A040603199B
:100EE80000340406702F782F83160516851608001F
:02400E0032FF7F
:104200000000010002000300410062004800650058
:104210006C006C006F00FF00FF00FF00FF00FF005C
:00000001FF
